:020000040000FA
:1000000077696E5F636861740000000000000000A3
:1000100000000000030000000002000014000000C7
:10002000016070474DF6A15CC0F60D0C604744F6C8
:10003000E55CC0F6020C604741F21B5CC0F60D0C9B
:10004000604747F6E77CC0F60E0C604744F65F5CFD
:10005000C0F6020C60474FF21D0CC0F60D0C604755
:100060004CF28F0CC0F60D0C60474FF2FF1CC0F62F
:100070000D0C60474EF63F4CC0F60D0C604747F63E
:100080001B7CC0F60E0C60474FF2995CC0F60D0C5D
:1000900060474CF23B3CC0F60D0C60474CF2D53C3F
:1000A000C0F60D0C60474BF6B93CC0F60D0C60472E
:1000B00048F6255CC0F60D0C60474CF2913CC0F64A
:1000C0000E0C604741F24F5CC0F60D0C60474EF6D7
:1000D000651CC0F60D0C60474FF25F5CC0F60D0C5E
:1000E00060474DF64F5CC0F60D0C604748F6B75CB4
:1000F000C0F60D0C604748F2492CC0F60D0C604765
:1001000044F6851CC0F6020C60474FF6B15CC0F6A1
:100110000D0C60474AF2834CC0F60D0C604748F264
:100120008D5CC0F60D0C604747F61B7CC0F60E0CCC
:10013000604747F6697CC0F60E0C604744F6297CA0
:10014000C0F6020C60474DF2875CC0F6020C6047B7
:100150004BF2010CC0F6020C60474BF2090CC0F6E2
:10016000020C604745F6BB6CC0F6020C604745F6D2
:100170006B7CC0F6020C604745F68F2CC0F6020C73
:10018000604745F6791CC0F6020C604748F2392CEE
:10019000C0F6020C604748F2073CC0F6020C60470C
:1001A00048F2174CC0F6020C604744F61F1CC0F61C
:1001B0000D0C604748F2835CC0F6020C604745F2C4
:1001C000977CC0F6020C604748F26D4CC0F6020CFA
:1001D000604748F2CD5CC0F6020C604744F6932CB1
:1001E000C0F6020C604740F2812CC0F6020C60475A
:1001F00040F2852CC0F6020C604748F6B31CC0F6EE
:100200000D0C60472DE9F04591B004460E46D4F838
:10021000B40DB04228D100200F901090D4F8A41D46
:10022000D1F8F42004F5E47151F822000FA900F090
:100230008FFC0FA904F5337000F02BFD012809D1C4
:1002400041F288306EA370A272A100902046FFF7A1
:10025000E9FE08E041F2883069A370A26DA1009028
:100260002046FFF7DFFEC8E0D4F8BC0DB04235D120
:100270000127D4F8C00D28B1D4F8C00DB0F8F400AF
:10028000401C87B2D4F8B00D00F1F4054FF4807033
:10029000FFF7CDFE804641462846FFF7CDFE40469B
:1002A000FFF7CFFE824653464246394604F5337087
:1002B00000F004FF4046FFF7C9FE02235AA2394668
:1002C00004F5337000F0FAFED4F8B01D01F1F40229
:1002D0007321D4F8AC0DFFF7BEFE8EE0D4F8B80D54
:1002E000B042C0D1D4F8C401022814D1D4F8A80D6A
:1002F00000F1F40104F5337000F049FFD4F8A80DC3
:10030000D0F8D01088470020C4F8A80D04F5337049
:1003100000F05AFF13E0D4F8C40101280FD104F60D
:10032000A4542068D0F8D0108847002020602069AD
:10033000D0F8D010884700202061A4F6A4540121F1
:1003400004F5337000F0EFFED4F8B80DD0F8D010FB
:1003500088470020C4F8B80D32212046FFF780FE00
:10036000A568E768C820A5F10A0305221146009098
:100370002046FFF77AFEC4F8AC0D2820A5F1A003B3
:10038000CD22052100902046FFF774FEC4F8B00D81
:1003900020222649794409A8FFF771FE09A8049094
:1003A000801D05900CA80690801D07900FA808904E
:1003B00028206421CD22A5F19B03CDE900210290E4
:1003C000052204A92046FFF75FFEC4F8C00D1920DE
:1003D0003221A5F13702D223CDE9001000212046B9
:1003E000FFF757FEC4F8BC0D11A1D4F8BC0DFFF700
:1003F00055FE2046FFF757FE00BF11B0BDE8F0855F
:10040000C8B7B6A800000000C1ACBDD3B3C9B9A637
:1004100000000000CCE1CABE00000000C1ACBDD3AA
:10042000CAA7B0DC000000000D0A00004414000060
:10043000B7A2CBCD000000002DE9F04106460C46E6
:1004400001F05AF907464FF00008002520680A28F5
:1004500043D2DFE800F04209050D42304222422C2F
:10046000304600F0C1F839E0304600F03DF835E0A4
:10047000E568287C00F0010000B900BF287C00F08E
:10048000080020B13046D6F8D010884726E0286909
:1004900010B13046FFF707FE20E0D4F80C80D8F802
:1004A0000800032800D100E000BF00BF16E030467E
:1004B00000F028F812E0E068012802D0022809D1F3
:1004C00000E008E02069012803D130466168FFF7A9
:1004D00099FE00E000BF00BF00E000BF00BF38464B
:1004E00001F024F9BDE8F0812DE9F0410446002532
:1004F0000026A768D4F80C802046FFF7D9FDBDE898
:10050000F08100002DE9F84F064600BF06F5337074
:1005100000F0E1FB0028F9D14FF48070FFF787FD70
:1005200004460025002756E04FF00008394606F53E
:10053000337000F04BFC8046B8F1000F4AD038E031
:100540000020605500BF11E0691E091A0DD4691E14
:10055000091A615C0D2904D0691E091A615C0A2917
:1005600003D10022691E091A6254401C0328EBDBE8
:10057000D6F8AC0DE8B14FF48070FFF758FD824615
:10058000B8F8062017A15046FFF797FD5046FFF731
:1005900058FD00EB0A0B59462046FFF793FD5246E3
:1005A0007221D6F8AC0DFFF756FD5046FFF74EFD11
:1005B00000BF0A200090B8F806106423224606F512
:1005C000337000F088FC05460DB1012000E00020EA
:1005D0000028B5D17F1C052FA6DB2046FFF736FD8E
:1005E000BDE8F88F25643A002DE9FE4F0446A66861
:1005F000E56804F5337000F086FC04F5337000F014
:10060000B3FC70B941F2883065A367A26BA100907A
:100610002046FFF707FD2046D4F8D0108847BDE8F4
:10062000FE8F94F8C00131287CD10120C4F8C401A8
:1006300004F5337000F090FD2346624A7A4462A1CB
:100640002046FFF744FD06EB46082F462D205A2191
:10065000CDE90010E81705EB907083104FEAE870C1
:1006600008EB9070821000212046FFF712FDC4F8BD
:10067000B40D5AA1D4F8B40DFFF710FD06EB4608EF
:1006800005EB45072D208221CDE90010F81707EB77
:10069000907083104FEAE87008EB90708210002190
:1006A0002046FFF7F6FCC4F8B80D4EA1D4F8B80DFB
:1006B000FFF7F4FC06EB4600052190FBF1FA2F460C
:1006C0004FEA45084FEAE87008EB90708010E91790
:1006D00005EB9171891014230022CDE9001A0290D4
:1006E00004F5E4712046FFF7CFFCC4F8A40D002701
:1006F00012E004F5E47050F82780803050F82700AD
:10070000007818B104F5127050F827804146D4F8EB
:10071000A40DFFF7E1FC7F1CD4F8C802B842E8DC66
:1007200039E0FFE794F8C001322834D10220C4F840
:10073000C401B04605EB45072D208221CDE900100C
:10074000F81707EB9070831006EBD8704210002169
:100750002046FFF79EFCC4F8B80D22A1D4F8B80DCE
:10076000FFF79CFCB2462F46B346A846E81705EBB8
:1007700090708010009006EBDB704310E81705EBDB
:1007800090708210F01706EB907081102046FFF7F2
:1007900071FCC4F8A80D2046FFF785FC00BF3EE7BA
:1007A000C8B7B6A800000000C0B6D1C0C4A3BFE956
:1007B000B8B4CEBBCAA7B0DCA3A10000B4EDCEF3A1
:1007C00000000000AD0F0000D5FDD4DAC9A8C3E8D1
:1007D000C0B6D1C0B4D3BBFA2E2E2E00C1ACBDD34F
:1007E00000000000CFC2D2BBB2BD00007CB5044601
:1007F000002611A012A314A216A100902046FFF714
:1008000070FC08B9312600E03226D4E90201002349
:100810001A46CDE900011946204600F01FF80546AA
:1008200085F8C06104F13C012846FFF75FFC2846CB
:10083000FFF761FC00207CBDB4D3BBFA00000000D0
:10084000D6F7BBFA00000000C7EBD1A1D4F1BDC7B9
:10085000C9AB0000CCE1CABE000000002DE9FE4F8C
:1008600007460E4690469A46DDF830B00EB9234E44
:100870007E4440F6C450FFF7DAFB0446002C39D022
:1008800040F6C45200212046FFF73AFC0D9843463B
:1008900032463946CDE900AB02902046FFF735FCE1
:1008A00020B92046FFF7D2FB002423E014A06061AA
:1008B0000120606616487844C4F8D0000020A06388
:1008C000144860631020FFF725FCC4F8BC01002524
:1008D0000EE01420FFF7ABFB04F5E47141F82500AE
:1008E0001420FFF7A4FB04F5127141F825006D1CDC
:1008F000202DEEDB2046BDE8FE8F0000C5FBFFFF8C
:1009000057494E5F43686174537472756374000095
:100910005F000000ACC1D70070B5044600F0ECFEEB
:10092000064600250CE004F5E47151F82500FFF7B8
:100930008DFB04F5127151F82500FFF787FB6D1C44
:10094000202DF0DB04F5337000F00EFBD4F8BC0171
:10095000FFF7E0FB2046FFF7E2FB304600F0E6FE43
:1009600070BD0146FF20302904DB392902DCA1F1EA
:100970003002D0B2412904DB462902DCA1F1370262
:10098000D0B2704710B500F063FC002010BD2DE917
:10099000F04D04460E4617469846DDE908AB207830
:1009A000FF2803D04FF0FF30BDE8F08D701E205CB3
:1009B000FC2802D04FF0FF30F6E74FF0FF35721EF3
:1009C000FB21601C00F003FE0546681C30B3BAF141
:1009D000000F02D0FB208AF80000B8F1000F05D00C
:1009E0002946601C00F0B4FEC8F800000FB1601C7E
:1009F00038600A9840B1F21E511B621C2A44501CF8
:100A000000F0A6FE0A990860BBF1000F04D0601C3C
:100A10002844401CCBF800000020C5E7721EFA21D4
:100A2000601C00F0D4FD0546681C30B3BAF1000F1D
:100A300002D0FA208AF80000B8F1000F05D029464C
:100A4000601C00F085FEC8F800000FB1601C386023
:100A50000A9840B1F21E511B621C2A44501C00F03F
:100A600077FE0A990860BBF1000F04D0601C28448F
:100A7000401CCBF80000002096E74FF0FF3093E7D2
:100A8000F8B5054600200090002400260EE09DF8F1
:100A90000000FF2800D101261EB19DF80000285556
:100AA000641C9DF80000FC2800D104E0684600F0BA
:100AB000E3FB0028EBD000BF9DF80000FC2801D12B
:100AC0002046F8BD4FF0FF30FBE710B500F0DEFB2D
:100AD000002010BD70B505460E46002403E0285DD9
:100AE00000F048FC641CB442F9DB002070BD00003B
:100AF0002DE9F04105460C461646FF2013494944AE
:100B0000087008464570FD20887004B14EB9FC207D
:100B10000E494944C87004210C484844FFF7DAFFE5
:100B200011E0324609494944C91C204600F035FD10
:100B30000746FC21F81C054A4A441154391D104649
:100B4000FFF7C8FF00BF0020BDE8F08144020000AD
:100B50002DE9F04706460F463546B8460024A24622
:100B600017E02878FFF7FDFE8246BAF1FF0F0FD09D
:100B700008EB6400007804F0010109B1002100E0F5
:100B800004210AFA01F1084308EB64010870641CAF
:100B90006D1C28780028E4D12046BDE8F08730B5E8
:100BA00002460B460BB9002030BD002418E0C4EB10
:100BB000041000EBC00502F1080000EB8501C888B5
:100BC00068B9D2F8B45A0D60B2F8B80A8880CB8000
:100BD000012088605068401C50600120E4E7641CDC
:100BE000052CE4DB0020DFE72DE9F04D04468B46C1
:100BF00017469846DDF824A000BFD4F8B00A0128B3
:100C00000EDAD4F8B00A00EBC00101EB001104F6D3
:100C100094200D18D4F8B00A401CC4F8B00A23E0A0
:100C2000D4F8B00A401E00EBC00101EB001104F63D
:100C300094200D18002612E0721C02EBC20303EB95
:100C4000021304F69422991806EBC60202EB06136F
:100C500004F6942298181922FFF766FA761CD4F845
:100C6000B00A401EB042E7DC2F703A465946681C75
:100C7000FFF75AFA781C054485F800806D1C85F84A
:100C800000A05246681C0899FFF74EFA0120BDE803
:100C9000F08DF8B504460D4604F6BA260020009003
:100CA000062229462120FFF723FF6A4631462046C7
:100CB00000F0A4F801280CD13078012809D104F5FE
:100CC00028602968C4F8B41AA988A4F8B81A0120C1
:100CD000F8BD0020FCE730B5A1B005460024642132
:100CE00008A8FFF726FA08A8FFF7CAFE0446601C0A
:100CF00028B908A8FFF722FA002021B030BD002053
:100D00000790069005900490039006A807A903AAEF
:100D100004ABCDE90021029005AA214608A8FFF7FF
:100D200036FE401C20B908A8FFF708FA0020E4E7C7
:100D30009DF80C00FB280BD1DDE90610CDE9000180
:100D40009DF80C302846DDE90421FFF74DFF1AE03D
:100D50009DF80C00FA2816D105980078012806D1D4
:100D6000079842880188284600F0E9F80BE00598CA
:100D70000078022807D10698831E07980188821CF4
:100D8000284600F020F90120B7E710B502460B46CF
:100D90000BB9002010BD002114E0C1EB011000EBE5
:100DA000C00402F1080000EB8400C088984208D11A
:100DB000C1EB011000EBC00402F1080000EB84005D
:100DC000E8E7491C0529E8DB0020E3E7024605299E
:100DD00012DAC1EB011000EBC00302F1080000EBD6
:100DE0008300C08840B1C1EB011000EBC00302F1E9
:100DF000080000EB830070470020FCE77CB5064646
:100E00000C46154600BF3046FFF765FF00231A4623
:100E100019463046CDE9004500F004F80028F2D02C
:100E200001207CBD2DE9F04D05460F4690469A46BF
:100E3000DDF820B0D5F8B00A00284AD005F6942491
:100E400027B12278611C3846FFF76EF9B8F1000F20
:100E500002D02078C8F80000BAF1000F04D0207842
:100E6000401C205C8AF80000BBF1000F08D02078FD
:100E7000801C225C2078C01C01195846FFF754F9E9
:100E8000099820B12078801C215C09980160002617
:100E900012E0721C02EBC20303EB021305F694226C
:100EA000991806EBC60202EB061305F69422981871
:100EB0001922FFF739F9761CD5F8B00A401EB04266
:100EC000E7DCD5F8B00A401EC5F8B00A0120BDE83D
:100ED000F08D0020FBE72DE9F047074688461446D1
:100EE0001D46DDF820A041463846FFF74EFF064676
:100EF0003EB153462A462146304600F00EFBBDE87F
:100F0000F0870020FBE770B50446FFF7DEFD69209F
:100F1000207000206060C4F8B00A00250AE0C5EB2C
:100F2000051101EBC10204F1080101EB820000F0A0
:100F3000E7FA6D1C052DF2DBFFF724FD70BD70B5DF
:100F400005460E461446012C04D131462846FFF7CB
:100F500026FE07E024B93146284600F050F901E0AA
:100F6000002070BD0120FCE7FEB5044604F6BA255A
:100F700000200290642600BF002211460320FFF7E4
:100F8000B7FD0220FFF7DFF82046FFF7A4FE02A816
:100F900000231A461946CDE900502046FFF742FFCC
:100FA0000298012809D12878012806D16420FFF78A
:100FB000CAF8FFF7E7FC0120FEBD3000A6F10106EC
:100FC000DAD100BFF8E72DE9F0410746884614461C
:100FD0001D4641463846FFF7D8FE064636B12A463A
:100FE0002146304600F0C2FABDE8F0810020FBE760
:100FF0002DE9F84307460D46144607F6BA260020A9
:1010000000902060002211462320FFF771FD40F67A
:10101000AC50FFF798F850E06A4631463846FFF783
:10102000EDFE012847D10098012806D1307801282B
:1010300001D1BDE8F8830020FBE7009807283CDBDE
:10104000206800EBC00000EB4000284431680160DC
:10105000B1888180B07940B2216801EBC10101EB18
:101060004101294488710098072818DD0098A0F1F3
:101070000708216801EBC10101EB41012944C81DAA
:101080004246F11DFFF750F80021206800EBC00038
:1010900000EB40002844C01D00F8081007E00020C5
:1010A000216801EBC10101EB41012944C8712068AD
:1010B000401C206001E00020BBE7ADE72DE9F845CA
:1010C00082460F4690461C460AF6BA25002000903C
:1010D000002624E02F7038126870142C01DD1426CD
:1010E00000E0264632464146A81CFFF71DF8B21C18
:1010F00029460720FFF7FCFC6A4629465046FFF7C1
:101100007DFE012807D12878012802D12CB9BDE83D
:10111000F8850020FBE70020F9E7A41BB044002C71
:10112000D8D10020F3E733B581B0054605F6BA24DF
:1011300000200090012202A90620FFF7D9FC6A4690
:1011400021462846FFF75AFE012803D120780128BE
:1011500000D13EBD0020FCE738B5044604F6BA25B0
:1011600000200090002211462020FFF7C1FC6A46B3
:1011700029462046FFF742FE012806D1287801289B
:1011800003D168202070012038BD0020FCE7F8B5AD
:1011900004460D4604F6BA26002000902846FEF7C5
:1011A00050FF07463A4629460120FFF7A1FC6A4650
:1011B00031462046FFF722FE012803D1307801286E
:1011C00000D1F8BD0020FCE738B5044604F6BA2586
:1011D00000200090002211461020FFF789FC6A468B
:1011E00029462046FFF70AFE012806D12878012863
:1011F00003D173202070012038BD0020FCE72DE9C9
:10120000F04105460E4616B90020BDE8F0810027E2
:1012100019E0C7EB071000EBC00105F1080000EB77
:101220008104E088B0420DD10020E080A060206001
:10123000A08004F10C0000F0AFF86868401E686000
:101240000120E2E77F1C052FE3DB0020DDE7000043
:1012500010B5FEF77DFF044600200649494448606A
:101260008860C860086148612046FEF776FF00206C
:1012700010BD00002C00000010B5044621460248B5
:10128000484400F0B0F810BD2C00000000B587B055
:1012900001210846FEF766FF01211020FEF767FFD7
:1012A000072209212F48FEF767FF07220A212D4850
:1012B000FEF762FF00208DF81A0001208DF81B0058
:1012C00002208DF818000002059002208DF8190008
:1012D00005A92448FEF755FF00208DF81A000220CA
:1012E0008DF818004002059005A91E48FEF749FF39
:1012F0001D48FEF74BFF4FF4E13001900020ADF8A0
:101300000800ADF80A00ADF80C00ADF810000C2094
:10131000ADF80E0001A91448FEF73DFF0121124867
:10132000FEF73EFF114979442520FEF73EFF0122DA
:1013300040F225510C48FEF73DFF25208DF80000B6
:1013400000208DF8010001208DF802008DF80300C7
:101350006846FEF734FF4FF40070054949440860C1
:1013600007B000BD00000240001001405B04000017
:101370002C00000010B5044621460648FEF724FF65
:1013800000BF80210348FEF724FF0028F9D0002089
:1013900010BD000000100140014600204860886038
:1013A000C860704730B502460B46916854680BE040
:1013B00002F11000405C984201D1012030BD491C6F
:1013C0001068884200DC00212000A4F10104EFD164
:1013D00000BFF3E710B504464FF4007020602046CC
:1013E000FFF7DAFF10BD2DE9F04104460D464FF03E
:1013F000FF36FEF7ADFE07462069C8B16068B8B198
:1014000004F11800A168405C28706068401E6060AC
:101410002878FC2802D12069401E2061A068401C69
:10142000A0602168A068884201DB0020A06000263F
:101430003846FEF792FE3046BDE8F081024650681D
:1014400090B102F110009368C05C08705068401EB3
:1014500050609068401C906013689068984201DB6F
:1014600000209060012070470020FCE72DE9F0414A
:1014700004460D464FF0FF36FEF76AFE0746FF2D85
:1014800001D101206061D4E90010884219DA606955
:10149000B8B104F11800E16845546068401C606010
:1014A000FC2D04D12069401C206100206061E068AF
:1014B000401CE0602168E068884201DB0020E060B9
:1014C00000263846FEF749FE3046BDE8F081024668
:1014D000D2E90030984211DA02F11000D368C15409
:1014E0005068401C5060D068401CD0601368D068C1
:1014F000984201DB0020D060012070470020FCE70B
:1015000010B504460020E080A0602060A08004F1B7
:101510000C00FFF75FFF012010BD2DE9F8430546E1
:10152000884616461F46394605F10C00FFF73AFF7C
:1015300010B90020BDE8F88300240020009014E0DA
:10154000694605F10C00FFF779FF08B92046F1E77D
:101550002EB19DF8000008F80400761E641C9DF86A
:101560000000B84201D12046E4E7E9E72DE9F04167
:1015700005460E461746002409E0315D05F10C00D2
:10158000FFF7A5FF10B92046BDE8F081641C3800C4
:10159000A7F10107F1D12046F6E730B503460C4626
:1015A0000FE01878F02804DA18780870491C5B1CE2
:1015B00007E0F0200870491C1878F0380870491CC2
:1015C0005B1C1000A2F10102EBD1081B30BD10B56D
:1015D0000346002004E01C5C8C4200D110BD401C7E
:1015E0009042F8DB4FF0FF30F8E700002DE9FF4DA7
:1015F000074600F081F883463E464FF45870FEF7E8
:1016000016FD054606F532722946101DFFF7F0FC5F
:10161000002455E006F5E47050F8248004EBC40083
:1016200000EB40002844407904EBC40101EB410188
:101630002944097904EBC40202EB42022A44D2781D
:1016400004EBC40303EB43032B449B78CDE9003246
:10165000CDE9021004EBC40000EB400028444378BD
:1016600004EBC40000EB40002A5C1CA14046FEF7DE
:1016700024FD04EBC40000EB40002844C079C0B155
:1016800006F5127050F8248004EBC40101EB41010F
:101690002944C81DFEF7D5FC00F1010A04EBC40083
:1016A00000EB40002844C11D52464046FEF796FD1F
:1016B00005E0002106F5127050F824000170641C4A
:1016C000D6F8C802A042A5DC2846FEF7BFFC584663
:1016D00000F02CF8002004B0BDE8F08D2530325821
:1016E000253032582530325825303258253032587E
:1016F000253032580000000010B5FEF774FD044696
:10170000034878440068FEF773FD204610BD0000D2
:10171000D200000010B5FEF766FD044621460248DF
:101720007844FEF77DFC10BDB400000010B50446FF
:101730002046FEF75DFD10BD70B50546FFF7EAFFD8
:10174000FEF75BFD04462046FFF750F8002070BD11
:1017500030B503460C4619461A460FE00878F028C3
:1017600005DA08781070521C491C641E06E00878DF
:101770004D7828441070521C891CA41E002CEDD1F9
:10178000D01A30BD70B5FFF7B7FF044600250F48EB
:10179000008800F0200078B10C488088C5B2294646
:1017A0000B484844FFF762FE0A4848440068401C62
:1017B00008494944086005E004480088C5B2034868
:1017C0008088C5B22046FFF7B1FF70BD0010014010
:1017D0002C0000000800000000000000CDA8B5C0EB
:1017E0003100CDA8B5C03200CDA8B5C03300CDA81A
:1017F000B5C03400CDA8B5C0350000000000000021
:081800000100000000000000DF
:0400000500001739A7
:00000001FF
